:020000040000FA
:02000000D32EFD
:08000800FF000308FE000A08D6
:10001000FC008312031323308100A20A073022025E
:100020000318A2012114A30F1828A40F1828A11443
:100030005408003E03193128451C2F280516792342
:100040000130832300001E30A500051207308323F2
:10005000051606308323A50B25280512532879237E
:1000600033286E236A231830A6002830FB00FA01DB
:10007000220803195C200130220203196820023093
:100080002202031974200330220203198020043055
:10009000220203198C200530220203199820063011
:1000A00022020319A42085010B117C088A007E0816
:1000B0008300FF0E7F0E0900B020A60B5C281022E3
:1000C000B0201622B0202422B0207223B0200800D5
:1000D000E120A60B68281022E1201622E12024222C
:1000E000E1207223E12008001221A60B74281022BF
:1000F0001221162212212422122172231221080019
:100100004321A60B802810224321162243212422BA
:1001100043217223432108007421A60B8C2810224E
:100120007421162274212422742172237421080060
:10013000A521A60B98281022A5211622A52124224C
:10014000A5217223A5210800D621A60BA4281022E0
:10015000D6211622D6212422D6217223D6210800A8
:100160000000000001082802031CFB14000000002E
:1001700001082902031C7B150000000001082A0267
:10018000031C7A140000000001082B02031CFA145F
:100190000000000001082C02031C7A15000000007A
:1001A00001082D02031C7A16831603137B088500B1
:1001B0007A0887008312031301308500003087001E
:1001C0000800280EA70001082702031C7B1400006A
:1001D000000001082E02031C7B150000000001082E
:1001E0002F02031C7A140000000001083002031CD7
:1001F000FA140000000001083102031C7A15000007
:10020000000001083202031C7A16831603137B08D0
:1002100085007A08870083120313023085000030BE
:1002200087000800290EA70001082702031C7B1481
:100230002E0EA70001082702031CFB14000000007B
:1002400001083302031C7A14000000000108340284
:10025000031CFA140000000001083502031C7A1583
:100260000000000001083602031C7A1683160313EF
:100270007B0885007A088700831203130430850009
:100280000030870008002A0EA70001082702031C7F
:100290007B142F0EA70001082702031CFB14330E4A
:1002A000A70001082702031C7B15000000000108BD
:1002B0003702031CFA140000000001083802031C76
:1002C0007A150000000001083902031C7A16831613
:1002D00003137B0885007A0887008312031300301C
:1002E00085000130870008002B0EA70001082702B7
:1002F000031C7B14300EA70001082702031CFB140B
:10030000340EA70001082702031C7B15370EA70037
:1003100001082702031C7A140000000001083A02B9
:10032000031C7A150000000001083B02031C7A162A
:10033000831603137B0885007A0887008312031352
:10034000003085000230870008002C0EA70001084D
:100350002702031C7B14310EA70001082702031C8F
:10036000FB14350EA70001082702031C7B15380E6D
:10037000A70001082702031C7A143A0EA7000108FF
:100380002702031CFA140000000001083C02031CB1
:100390007A16831603137B0885007A088700831278
:1003A0000313003085000430870008002D0EA700DD
:1003B00001082702031C7B14320EA7000108270244
:1003C000031CFB14360EA70001082702031C7B1533
:1003D000390EA70001082702031C7A143B0EA70060
:1003E00001082702031CFA143C0EA700010827028B
:1003F000031C7A15831603137B0885007A0887008F
:100400008312031300308500103087000800831624
:1004100003137B0885008312031320308500080036
:1004200003103D0DC6001D22C900080003103D0D3C
:10043000013EC6001D22CA00080002308A0046089C
:10044000283E03188A0A820049088A004A08820066
:10045000023468340234733402347B34023483341B
:1004600002348B340234933402349B340234A73484
:100470000234AB340234B7340234BB340234C734F0
:100480000234CB340234D7340234DB340234E73460
:100490000234EB340234F7340234FB3403340734CF
:1004A00003340B340334173403341B34033427343C
:1004B00003342B340334373403343B3403344734AC
:1004C00003344B340334573403345B34033467341C
:1004D000C4013030C8003F18702A0630BD00692BB7
:1004E0000130BD00692B3F18782A0030BD00692B10
:1004F0000230BD00692B3F18802A0030BD00692BF7
:100500000330BD00692B3F18882A0430BD00692BD9
:100510000330BD00692B3F18902A0030BD00692BC5
:100520000530BD00692B3F18982A0730BD00692BA4
:100530000030BD00692B3F18A52A00304807031979
:10054000A32AC80B692B4414692BBD01692B3F08F2
:10055000C300BD0A692B43083F06031DB12ABD0134
:10056000692B3F1842103F1C4214BD0A692B3F08FB
:10057000C300BD0A692B43083F06031DC12ABD0104
:10058000692B3F1841123F1C4116BD0A692B3F08D9
:10059000C300BD0A692B43083F06031DD12ABD01D4
:1005A000692B3F18C1113F1CC115BD0A692B3F08BB
:1005B000C300BD0A692B43083F06031DE12ABD01A4
:1005C000692B3F1841113F1C4115BD0A692B3F089B
:1005D000C300BD0A692B43083F06031DF12ABD0174
:1005E000692B3F18C1103F1CC114BD0A692B3F087D
:1005F000C300BD0A692B43083F06031D012BBD0143
:10060000692B3F1841103F1C4114BD0A692B3F085C
:10061000C300BD0A692B43083F06031D112BBD0112
:10062000692B3F18C0123F1CC016BD0A692B3F083A
:10063000C300BD0A692B43083F06031D212BBD01E2
:10064000692B3F1840123F1C4016BD0A692B3F081A
:10065000C300BD0A692B43083F06031D312BBD01B2
:10066000692B3F18C0113F1CC015BD0A692B3F08FC
:10067000C300BD0A692B43083F06031D412BBD0182
:10068000692B3F1840113F1C4015BD0A692B3F08DC
:10069000C300BD0A692B43083F06031D512BBD0152
:1006A000692B3F18C0103F1CC014BD0A692B3F08BE
:1006B000C300BD0A692B43083F06031D612BBD0122
:1006C000692B3F1840103F1C4014BD0A692BBD0127
:1006D000471408004410851E441408003F10851973
:1006E0003F1408003E083D02031C782B3D08BE0065
:1006F00008004510D4030310D30CD20CD10CD00C3D
:10070000031845140800CB00CB0B842B0800D10143
:10071000D201D301A030D000CE094E1C51144E1886
:10072000D1144C1E51154C1AD115CC1D5116CC1993
:10073000D1164C1D51174C19D117CC1C5214CC1882
:10074000D2144C1C52154C18D215CD1E5216CD1A6F
:10075000D2164D1E52174D1AD217CD1D5314CD1956
:10076000D3144D1D53154D19D315CD1C5316CD184B
:10077000D3164D1C53174D18D3172130D400080041
:10078000D501D6010830D7000310D90CD60DD50DF0
:10079000D80CD60DD50DD70BC42B0800DA000000FD
:1007A000DA0BCF2B0800E30A63081A3C0319E301B4
:1007B0006308CF000800E3036308013E031DE32B39
:1007C0001930E300CF0008004008E300CF00E63E08
:1007D000031CEE2B1930E3026308E72B0800DB0053
:1007E0002110211CF12BDB0BF02B0800630AE50024
:1007F000D800D901C0235508E5005608E600E701F6
:10080000E8010C30E900711C082CE809FC30E90013
:10081000FF301525E501E601E70101301525080047
:100820006308031D1E2C03015824DE00F101DE1BAA
:1008300071145E08031D322CD323102C0730DC000A
:100840000C30DD000310630DF9008B1305278B17A7
:10085000DF000314630DF9008B1305278B17DD00F0
:100860005F08DC0008006308031D392C7908582450
:10087000432C8B130A08E00079080527E100600883
:100880008A0061088B17F90A0800831603139C1865
:10089000472C8B131C1579089B0078089A0055305B
:1008A0009D00AA309D009C148B178312031308002F
:1008B0008B13831603139C185B2C1C119B009C1339
:1008C0001C141A08831203138B1708000301582401
:1008D000E200E21F6E2CE213F101702CE21771149A
:1008E000F9016208F8004524F623F62308001024D5
:1008F000F9013324E400E4133324F000F00A332434
:10090000F200471C9F2C07304102031D8A2CE42370
:10091000C701772CC108031D9F2C2030400203190A
:10092000D323213040020319DB2300304002031996
:10093000E3010C30400203196624C701772C441CE4
:10094000AB2CF623F623441CAB2CD323F623F6233F
:100950004418A52C772C093064020319CA240C30E2
:1009600064020319E9240D3064020319F6245408C3
:10097000003E031DC72CA11CC72CA110711CC22C4A
:10098000D323772C0730CC004F08CD008723F20B00
:10099000812C772C3324E5003324E6003324E70050
:1009A0003324E8003324E90003306905F300F30A37
:1009B000F30DF30D70081525F30BDA2C0800740DF8
:1009C000740D741A013AF41A013AF419013AF40058
:1009D0000800DF24E800DF24E500DF24E700DF244F
:1009E000E600DF24E9007008152508003324E5003F
:1009F0003324E6003324E7003324E8003324E900FD
:100A00003324EA003324EB003324EC003324ED00DC
:100A10003324EE000F306E05F300F30AF30DF30DEF
:100A20007008A025F30B102D0800EF00AE01AF01F8
:100A3000B301B401B701B801B901BB01AB01AA010F
:100A4000A901A801B101B001B501B601AD01AC0128
:100A5000B201BA01BC01F030E718A804F030E71980
:100A6000A904F030E71AAA04F030E71BAB04F03019
:100A7000E91AAC04F030E91BAD040F306718A80484
:100A8000F030E51BAE04F030E51AAF04F030E81AA0
:100A9000B004F030E81BB104F030E919B2040F30B3
:100AA0006719A9040F30651BAE04F030E519B304D3
:100AB000F030E518B404F030E819B504F030E81867
:100AC000B6040F30671AAA040F30651AAF040F304E
:100AD0006519B304F030E61BB704F030E61AB80429
:100AE000F030E619B9040F30671BAB040F30681AF9
:100AF000B0040F306518B4040F30661BB704F03033
:100B0000E618BB040F30691AAC040F30681BB1043F
:100B10000F306819B5040F30661AB8040F30691B1E
:100B2000AD040F306919B2040F306818B6040F30E5
:100B30006619B9040F306618BB046F08EF2308006C
:100B4000EF00AE01AF01B301B401B701B801B901C3
:100B5000BB01AB01AA01A901A801B101B001B50116
:100B6000B601AD01AC01B201BA01BC01A030E51B78
:100B7000AE074030651BAE070A30E51AAE070430F9
:100B8000651AAE07A030E519AF0740306519AF0709
:100B90000A30E518AF0704306518AF07A030E61B30
:100BA000B3074030661BB3070A30E61AB3070430B8
:100BB000661AB307A030E619B40740306619B407C7
:100BC0000A30E618B40704306618B407A030E71BF3
:100BD000B7074030671BB7070A30E71AB70704307A
:100BE000671AB707A030E719B80740306719B80788
:100BF0000A30E718B80704306718B807A030E81BB8
:100C0000B9074030681BB9070A30E81AB907043041
:100C1000681AB907A030E819BB0740306819BB074C
:100C20000A30E818BB0704306818BB07A030E91B7E
:100C3000AB074030691BAB070A30E91AAB07043039
:100C4000691AAB07A030E919AA0740306919AA0749
:100C50000A30E918AA0704306918AA07A030EA1B6D
:100C6000A90740306A1BA9070A30EA1AA90704300D
:100C70006A1AA907A030EA19A80740306A19A8071C
:100C80000A30EA18A80704306A18A807A030EB1B3E
:100C9000B10740306B1BB1070A30EB1AB1070430C3
:100CA0006B1AB107A030EB19B00740306B19B007D1
:100CB0000A30EB18B00704306B18B007A030EC1BFB
:100CC000B50740306C1BB5070A30EC1AB507043085
:100CD0006C1AB507A030EC19B60740306C19B6078E
:100CE0000A30EC18B60704306C18B607A030ED1BBC
:100CF000AD0740306D1BAD070A30ED1AAD0704306B
:100D00006D1AAD07A030ED19AC0740306D19AC0776
:100D10000A30ED18AC0704306D18AC07A030EE1B9C
:100D2000B20740306E1BB2070A30EE1AB207043029
:100D30006E1AB2076F08EF23080002303D02031C51
:100D40000301E5000030E60001301525441CB72EF4
:100D5000BE01BD015408003E031DB72EE501E601AA
:100D6000E609FF301525CC010C30CD008723471C48
:100D70009D2EC701F030E500E6017F301525E50125
:100D8000E6013F301525F030E500E6017F301525FE
:100D90004008E5004108E600FF301525FF30152525
:100DA000BE01BD019D2E85018101E301D401C20177
:100DB000C101C001C301BD01BE01C701A2010730CD
:100DC00099008316031382308100811395019516D3
:100DD00070308F04910183120313C4011D30F4009D
:100DE0008B168B17FF30E500E600E700E800E9000E
:100DF000FF301525E501E601E701E801E901FF30D3
:100E00001525441C772C66249D2E5C088A007908E1
:100E10005D0703188A0A82000734403407344034DF
:100E200007347F340734B4340734F33408340534DA
:100E300008343534083488340834A9340834B634D6
:100E40000834C8340834DF3409341E3409343034EB
:100E500009346F340934AE340934CF340934F034F2
:100E60000A349D340B343B340B34CF340B34F03420
:100E70000B34F3340C34AA340C34DF340D341E3408
:100E80000D343034063455345534553455345534D6
:100E900055345534553455345034AA34AA34AA3410
:100EA000AA34AA34AA34AA34AA34AA34A034FF3407
:100EB000FF34FF34FF34FF34FF34FF34FF34FF349A
:100EC000F034AA34AA34AA34AA34AA34AA34AA34EC
:100ED000AA34AA34A03455345534553455345534D5
:100EE00055345534553455345034003400340034BE
:100EF0000034003400340034003400340034093449
:100F000010340A34C0340C340034C3340C3420346C
:100F100012340134C3340C342034123401342434F8
:100F20009C3408344034843424349C3403340034F6
:100F3000303424349C3403340034303400340C34E2
:100F400003340034303418346C340434803448347E
:100F500018346C341034213402341834C034103452
:100F600021340234C3340C34093410340C3450347A
:100F700000340034803400341434003400348034BD
:100F8000003405340034003400342034013440345B
:100F900000340034203400345034003400348034C1
:100FA0000034143400340034803400340534003408
:100FB000023400340034013440340234003400344C
:100FC000003450340834003400340034143408340D
:100FD000003400340034053420340034403400340C
:100FE00001342034003409343034033441340434BF
:100FF0001034413400341034413404340434103497
:101000000434103441341034403409343034093459
:1010100040340034003400340034103400340134DF
:1010200000340034043400340434403400340034D8
:1010300000340034103410340134003410340034DF
:101040000434003400340034043440340034403478
:10105000403401340034003411340034003400349E
:101060000034043400340034003409343034103493
:10107000803400340034003400342034003402342E
:1010800000340034083400340834003400340234AE
:101090000034203400340034003480348034003490
:1010A0000034003422340034003400340034083476
:1010B000003400340034003400340034023400348E
:1010C00000340034003408348034003400340034F8
:1010D00020342034003400340034803400340034B0
:1010E0000034003400340434003400340034553407
:1010F0005C34553455345534FF34F034FF34FF3408
:10110000FF34003400340034003400340034003440
:101110000934303406345434003400345034043448
:10112000053440340034143404340034543400346E
:10113000053404340034053440340134443400347C
:1011400000345434003454344034003405344034D2
:10115000143409343034023466346634663400346E
:1011600000349934993499340034003409343034DB
:1011700003344834C4348C346D34BC34C4348C34BB
:101180004834DB346C348C344834C434B634DC3406
:10119000093430340434553455345534AA34AC341D
:1011A000AA34AA34AA34FF34F034FF34FF34FF34B5
:1011B00000340434003400340034553458340934D5
:1011C00030340C345534543400348234A034153463
:1011D000553400348234A034053455344034A034BE
:1011E000A034013455345034A03420340034553404
:1011F0005434A8342034003415345534A834003421
:10120000403405345534AA34003450340134553454
:101210002A3400345434003455342A34803455345C
:10122000003415340A3480345534403405340A34DB
:10123000A0345534503401340234A03409342034FD
:101240000334543405344034513444340534403488
:101250005434143454344034543405344534143440
:10126000093430340C340034003400340034043495
:10127000003400340034553450345534553455342A
:1012800000340034003400340034003400340034BE
:101290000034003400340834003400340034AA34FC
:1012A000A034AA34AA34AA34003400340034003400
:1012B00000340034003400340034003400340C3482
:1012C000003400340034FF34F034FF34FF34FF3492
:1012D0000034003400340034003400340034093465
:1012E00010340C3480340034003480340034203422
:1012F00000340034A0340034083400340034203486
:101300000034023400340034283400340034803493
:101310000034083400340034203400340A340034FB
:101320000034083400340234003400340234003411
:10133000023480340034003480340034803400348B
:10134000003420340034A034003400340834003435
:101350002034003400340234803420340934103412
:101360000634403404340034003400341034013482
:101370000034003400340434003440340034003489
:101380000134003410340034003400344034043468
:101390000034003400341034013400340034093493
:1013A0001034063400340034003480340034003407
:1013B0000034003420340034003400340034083465
:1013C000003400340034003402340034003400347B
:1013D00000340034803400340034003400342034CD
:1013E0000934073422340034193400340034003412
:1013F00000346234003401340034013402344034A7
:101400000A3400340434003440341034443410348A
:101410000034403440344834403400344034803464
:10142000903400340034413400342034003400342B
:101430009834003400340034003464340034003410
:1014400000340134A4340034003400340834083447
:10145000013490340034103409340234143400342C
:101460002034013404342834003440340134483406
:10147000083401340034013450340034583400341A
:101480000234003400346034003402340034003458
:1014900090340034013400340034203400340634F5
:1014A0004034003424340034103480342034043484
:1014B00000344034103444340434013400341134E2
:1014C0000834043404340034263400340434103432
:1014D00000340834003409348034003400340034DB
:1014E000063440340034003400341A3440340034BC
:1014F00000340034803480340034643400340034E8
:101500009034013484340434003410340234083408
:1015100018340034103404340134283400341034C6
:101520001034013440340034253480340034003425
:1015300000342634003400340034093407341F34B6
:101540008034003400340034003420340034023459
:10155000003400340834003408348034003400345B
:101560000034003420342034023400342034003479
:1015700008340034003400340834803400348034BB
:101580008034023400340034223400340034003417
:1015900000340834003400340034003400340034A3
:1015A000003400340034003400340034003400349B
:1015B0000434003400340034003404340034003483
:1015C0000034003411340034003400340034113459
:1015D00000340034003400344034403401340034EA
:1015E00000344034403401340034003400340034DA
:1015F00004344034003400340034043440340134C2
:101600000034103400340434013400341034003415
:101610000434003400340034103410340034003406
:1016200000341034103404340034043440340034B2
:1016300004340034043440340034103400340134B1
:1016400000340034103400340134003400344034A9
:1016500000340034003400344034003400340034AA
:1016600000340034003400340034003400340034DA
:10167000003400340034093404341D34C0340034E0
:101680000034003400343034003403340034003487
:10169000303400340334003400340C3400340C345F
:1016A000C03400340C3400340C34C03400340C34F6
:1016B00000340C34C034003400340034003430348E
:1016C00030340034003400343034303400340034EA
:1016D00000343034303400340034003430343034AA
:1016E00000340034003430343034033400343034C7
:1016F00000340C3403340034303400340C340334FC
:101700000034303400340C340334003430340034CA
:101710000C3403340034303400340C3400340034DE
:1017200000340C34C0340034003400340C34C03481
:101730000034003400340C34C0340034003400343D
:101740000C34C0340034003400340C34C034003461
:10175000C034C034033400340034C034C0340334E3
:1017600000340034C034C034033400340034333423
:101770000034003400340034333400340034003496
:1017800000340C34003400340034003400340034AD
:1017900000340034003400340034003400340934A0
:1017A000203406344234043420340034003400340D
:1017B000903409340034003400346034063400348A
:1017C00000348134083410340034003424340234BA
:1017D0004034003400341834013480340034003490
:1017E0000C3480340034093430342434543400341C
:1017F00000340034003401340034013450340034F7
:101800000034C0340C340C343C34003420342034E4
:101810000234803400340A3480340034003400341C
:1018200000340034003400340534403400340034D3
:10183000003410341034003414340034C0340C3408
:101840000034C3340C340034023402340034A03485
:1018500000340034A8340034003400340034003440
:101860000034003400345434003400340034013483
:1018700001340034053400340C340034C0343034C6
:10188000CC3420340034203480342034803400348C
:101890000A3400340034003400340034003400349E
:1018A0000034053440340034003400341034103433
:1018B000013440340034C0340C340C343C34023431
:1018C00000340234A0340034A8340034003400342E
:1018D0000034003400340034003400340034003468
:1018E00054340034003400340134013400345034B2
:1018F000C0340C340034C3340C342034203400346D
:10190000283400340A348034003400340034003485
:1019100000340034003400344034003405340034E2
:101920000034103400341034403410340C3400349B
:10193000C0343034CC340234023400340A3400343D
:101940000034AB340034003400340034003400344C
:1019500000340034093407340A34C0340C34003401
:10196000C3340C34203412340134C3340C342034E6
:101970001234013424349C34083440348434243404
:101980009C3403340034303424349C340334003425
:10199000303400340C3403340034303418346C34B4
:1019A00004348034483418346C3410342134023414
:1019B0001834C434103421340234C3340C340934A0
:1019C00007340C3450340034003480340034143480
:1019D00000340034803400340534003400340034E2
:1019E0002034013440340034003420340034503486
:1019F0000034003480340034143400340034803433
:101A000000340534003402340034003401344034EE
:101A100002340034003400345034083400340034CC
:101A200000341434083400340034003405342034D5
:101A3000003440340034013420340034093460343C
:101A40000434553455345534AA34AC34AA34AA3449
:101A5000AA34FF34F034FF34FF34FF34003404344C
:101A600000340034003455345834093410340C3404
:101A70005534503401340234A034553440340534E4
:101A80000A34A0345534003415340A3480345434C4
:101A9000003455342A3480345034013455342A34D7
:101AA0000034403405345534AA340034003415343D
:101AB0005534A8340034003455345434A834203418
:101AC000013455345034A034203405345534403476
:101AD000A034A0341534553400348234A034553445
:081AE000543400348234A034B8
:02400E00C430BC
:10420000090017002A00AA00AA00AA00AA00A80014
:1042100055005500550055005400FF00FF00FF00F9
:10422000FF00FC0000000000000000000000400053
:10423000000000000000000010000000000000006E
:104240000000040000000000000000000100000069
:10425000000000000000000040000000000000001E
:10426000000010000000000000000000040000003A
:10427000000000000000010000000000000000003D
:1042800000004000000000000000000010000000DE
:10429000000000000000040000000000000000001A
:1042A00001000000000000000000000040000000CD
:1042B00000000000000010000000000000000000EE
:1042C00004000000000000000000010000000000E9
:1042D000000000000000400000000000000000009E
:1042E000100000000000000000000400800000003A
:1042F000000000000000200000000000000000009E
:1043000008000000000000000000020000000000A3
:10431000000000000000800000000000000000001D
:104320002000000000000000000008000000000065
:10433000000000000200000000000000000000007B
:1043400080000000000000000000200000000000CD
:104350000000000008000000000000000000020053
:1043600000000000000000000000800000000000CD
:104370000000000020000000000000000000080015
:10438000000000000000000002000000000000002B
:10439000000000008000000000000000000020007D
:0A43A000000000000000000008000B
:00000001FF
